:03000000023F2894
:0C3F280078FFE4F6D8FD75816F023F6F52
:1013F9000A53746172743A20004950436F6E6E65E6
:1014090063745245510A004950436F6E6E656374A7
:10141900003E432C562C43432CC0E4E0EFF2E5F0A8
:1014290020D1E8EDEAEEEC49500A003E432C4D414B
:10143900432C25303262583A25303262583A2530E9
:101449003262583A25303262583A25303262583A77
:1014590025303262582C4D414320E0E4F0E5F10A91
:10146900003E432C5645522C20332E3120EEF220DB
:1014790025732025732CC2E5F0F1E8FF204950209F
:10148900ECEEE4F3EBFF0A004E6F762030332032A6
:101499003030370030383A35313A3231003E432C5A
:1014A9004C442C50524F473A202020202020202005
:1014B9002020202020202020202020202020202023
:1014C9002020202020202020202020202020202013
:1014D9002020202020202020202020202020202003
:1014E900202020202020202020202020202CC4E083
:1014F900F2E020EFF0EEF8E8E2EAE828F4E0E9EBC0
:10150900290A003E2A2C312CCEF1EDEEE2EDFBE565
:1015190020EFE0F0E0ECE5F2F0FB20F1E5F2E5E2A6
:10152900EEE3EE20E8EDF2E5F0F4E5E9F1E00A009A
:101539003E412C4130312C2562752E2562752E25B0
:1015490062752E2562752C495020E0E4F0E5F12002
:10155900E0E4E0EFF2E5F0E00A003E412C413032F0
:101569002C2562752E2562752E2562752E256275CC
:101579002C495020E0E4F0E5F120EEF1ED2E20F1C8
:10158900E5F0E2E5F0E00A003E412C4130332C253C
:1015990062752E2562752E2562752E2562752C4978
:1015A9005020E0E4F0E5F120F0E5E72E20F1E5F048
:1015B900E2E5F0E00A003E412C4130342C25627509
:1015C9002E2562752E2562752E2562752CCCE0F1CB
:1015D900EAE020F1E5F2E80A003E412C4130352CE1
:1015E9002562752E2562752E2562752E2562752C4C
:1015F900D8EBFEE70A003E532C4130362C256275A4
:101609002CC2F0E5ECFF20EEE6E8E42E20EAE2E861
:10161900F2E0EDF6E8E820282A3130ECF1290A0059
:101629003E2A2C312CC4EEEF2E20EFE0F0E0ECE561
:10163900F2F0FB20F1E5F2E5E2EEE3EE20E8EDF26F
:10164900E5F0F4E5E9F1E00A003E422C5330312C93
:101659002562752CC6E4E0F2FC20E7E0EFF0EEF13C
:10166900E020F1EEE5E4E8EDE5EDE8FF20EEF2201B
:10167900F1E5F0E2E5F0E00A003E422C5330322C6D
:101689002562752CCEE1ECE5ED20F120F1E5F0E2E3
:10169900E5F0EEEC20E1E5E720EAE2E8F2E0EDF63C
:1016A900E8E90A003E422C5330332C2562752CCFD1
:1016B900E5F0E5E7E0EFF3F1EA20EFF0E820EFEEFF
:1016C900F2E5F0E520F1E2FFE7E820F120F1E5F0AD
:1016D900E2E5F0EEEC0A003E422C5330342C256250
:1016E900752CCDE5F220EFE5F0E5E4E0F7E820E43C
:1016F900E8E0E3EDEEF1F2E8EAE820E220F1E5F0D6
:10170900E2E5F00A003E422C5330352C2562752C57
:10171900CAE0EDE0EB20F8E8F0EEEAEEE2E5F8E009
:10172900F2E5EBFCEDEEE3EE20EEE1ECE5EDE00AAF
:10173900003E532C5330362C253032625825303236
:10174900625825303262582530326258253032626B
:101759005825303262582C4D414320E0E4F0E5F140
:1017690020F8E8F0EEEAEEE2E5F8E0F2E5EBFCED70
:10177900EEE3EE20EEE1ECE5EDE00A003E454E44F5
:101789000A0044756D705820202020203030203008
:10179900312030322030332030342030352030367B
:1017A9002030372030382030392030412030422055
:1017B90030432030442030452030460A003A20008A
:1017C9000A0044756D7044202020202030302030DC
:1017D900312030322030332030342030352030363B
:1017E9002030372030382030392030412030422015
:1017F90030432030442030452030460A004572727B
:10180900206B657900526420656570726F6D0A00FE
:101819005264204D454D0A00526420436F64650AA5
:101829000044656275674950204F4E0A004465625D
:1018390075674950204F46460A00446562756755E9
:10184900736572204F6E0A0044656275675573654A
:1018590072204F46460A0044656275674D736720DA
:101869004F6E0A0044656275674D7367204F46469F
:101879000A00436F6E666967206C6F636B210A000B
:10188900577220656570726F6D0A00205361766525
:1018990020656570726F6D210A00457272204D4195
:1018A9004321004C6F61643E3E002A003C413031C7
:1018B9003D003C4130323D003C4130333D003C412C
:1018C90030343D003C4130353D003C4130363D002F
:1018D9004E4F4950004C494E4B434F4E54520054C1
:1018E90052415353004652004E4F4C494E4B00490A
:1018F9004E49004E4F4449414700003C21003C53AA
:1019090030313D003C5330323D003C5330333D00D3
:101919003C5330343D003C5330353D003C53303668
:101929003D00FF18D9FF18DEFF18E8FF18EEFF1871
:0A193900F1FF18F8FF18FCFF190376
:0648FD00010B000109009F
:1048BC00C2AFC28E438910758BFF758DB7D2ABD248
:0448CC008ED2AF22B7
:03001B00023D693A
:103D6900C0E0C083C082C0D0C2AFC28E758BFF7560
:103D79008DB720060675A61E75A6E10509D202E5CE
:103D89000B6002050BE50AD394014002150A050EE2
:103D9900E50E540F7050D20DE50E543F701AD20043
:103DA900907AF2E0601204F0E0D394B4400A908073
:103DB900007480F0C2AF80FE907AEDE0600204F0FA
:103DC900907569E0600214F0907AF3E0D3940140B1
:103DD90003E014F0300502050CE50DD394644004AA
:103DE900D2068002050DE508D3940140021508D2D8
:0C3DF9008ED2AFD0D0D082D083D0E03288
:10088100C291C290D2B5C20A7D027C007F07124894
:10089100508F26E526646060097D017F601248085B
:1008A100D20AE4FDFC7F0B1248508F26E52630E684
:1008B100097D04E4FF12482CD20A7D017C007F07E8
:1008C1001248508F26E5267008FD7FFF124808D296
:1008D1000A300A03126000C2AFC288C2A8C2AA7558
:1008E10089001241BD9077A6E0B4FA09A3E064CE75
:1008F1007003020981E4F526749E2526F582E4340D
:1009010077F583E4F00526E526B443EC9077A674E9
:10091100FAF0A374CEF0A374CCF09077AC740AF023
:10092100E4A3F0A304F0A3F09077B17403F0A374EF
:10093100CCF09077A274FFF0A3F0A3F0E4A3F090C1
:1009410077BD7405F0E4F526E5262401FFE433FEC6
:10095100749E2526F582E43477F583E0FD1248A3E1
:100961000526E526C3944340DFE4F5A775A61E7569
:10097100A6E1907FF0F0A3F09080007480F080FEFB
:10098100D2AF9077B17403F0A374CCF0E49077B058
:10099100F0123876EF6003122704C2B51224FFC2A9
:1009A100061245919077BDE0C3940350037403F0A0
:1009B100D20AC20CC20BD293200A077E137FF9120E
:1009C100395CE49079DDF01248BCC2AFA37408F041
:1009D10090771C7424F0E4A3F09077A6E090771E42
:1009E100F09077A7E090771FF09077A8E0907720BC
:1009F100F09077A9E0907721F09077AAE0907722A4
:100A0100F09077ABE0907723F0750A01E49079DFFD
:100A1100F0C207C208D2AF75A70775A61E75A6E179
:100A21001247E1200A19AF267E007D03123A3DE408
:100A3100FF123CBF7E777FDDE4FB7D01123B179007
:100A41007AF2E060037401F0E4907569F0A37455E3
:100A5100F0A37481F0E4F50CE4F50D907569E07094
:100A610003121F99907AF3E0B40111908000741081
:100A7100F0E4907AF3F0D20AD20BD20C908008E025
:100A8100F52630E405D2077410F0E52630E508D2EA
:100A9100099080087420F0E52630E608D20890809D
:100AA100087440F0E50CD394034023908002E4F0F5
:100AB100908001F0908000F0E50CD39406400FE4A3
:100AC100F50CC2039079DFF0750A0112459190800F
:100AD100A0E070031242B69080B8E0700312433078
:100AE1009080D0E0700312440F908000E0701330CA
:100AF1000710123772907799EFF0D39400400312E8
:100B01000026908002E07006908000E06005D2052A
:100B1100020A59C205E4F50C907569E06003020A06
:100B210059300912123137907799EFF0D394004080
:100B310005E0FF1248D0200803020CB8122FC29022
:100B41007799EFF07003020A599077DDE054BF24E2
:100B51007F7003020C1B147003020BF32402600369
:100B6100020C4E200A077E147F0212395C300E7986
:100B71002003769077B5E070069077B9E0605B90DE
:100B81007AE9E0FF9077B5E0B50724907AEAE0FED4
:100B91009077B6E0B50618907AEBE0FE9077B7E073
:100BA100B5060C907AECE0FE9077B8E06E602B9081
:100BB10077B9E06F7033907AEAE0FF9077BAE0B5E9
:100BC1000727907AEBE0FF9077BBE0B5071B907A9F
:100BD100ECE0FF9077BCE0B5070F9079DF7401F08E
:100BE100120021750A01020CB8907AE974FFF00233
:100BF1000CB8907AF2E060037401F0907AE1E0FFC2
:100C01009077DFE06F6003020CB8907AE1E004F0C6
:100C1100E4F50A9079DDF0020CB8300303020CB858
:100C21009077ACE07003020A59124904D203E4F54B
:100C31000A9079DDF0907AED04F0E4907AE0F0A387
:100C4100F0200A737E147F1012395C806A907AF268
:100C5100E060037401F03003529077DDE020E74B50
:100C61009077DFE0FF907AE0E0FE6F600D907AE828
:100C7100E07007EE146F703F8013907AE0E004F0AB
:100C8100907799E0FFD394044003124678907465FD
:100C91007482F0A37401F09077DFE0907467F07EC6
:100CA100747F657D0312423B020A59300E0920030D
:100CB10006907AE974FFF0200303020D6DE50A70D6
:100CC1006B124729EF60207E787FDD9078DEE0248B
:100CD10004FD12423B907AE8E06003020A599077E2
:100CE100BDE0F50A020A59907AEDE0D3943C403C0C
:100CF100907AE8E07036907AED04F090771BE0701E
:100D01002B1248EAE49078DDF0A37412F0907AE1B6
:100D1100E09078DFF0A374FDF090756C63A2019010
:100D210078E163A2017F12122BA9809B1248DFEFA9
:100D310060159074657483F0E4A3F07E747F657D23
:100D41000212423B020A59E50A64016003020A5990
:100D51009079DDE004F0E0C394055003020CC8C2B1
:100D610003E49079DFF0120021020A59E50A6401D7
:100D71006003020A599079DFE014604024FE603C70
:100D8100147003020E5524046003020A59E4F50CA1
:100D9100200E139079DF7404F09079DDE05401F0B6
:100DA100750A01020A59E49079DFF09079DD04F0C7
:100DB100750AC8907AE974FFF0020A59907AE9E05D
:100DC1007003020E449078DD7480F09078DF740136
:100DD100F0E4A3F0A304F0A37430F0A3747BF0E477
:100DE100F52674E42526F582E43478F583747DF0E4
:100DF10074E52526F582E43478F583E4F0E52624CC
:100E0100079078DEF07C7A7DE99077B1E0FAA3E093
:100E1100FB7F021240397E787FDDE5262409FD1231
:100E2100423B907AE8E0601B124904D203E4F50AE0
:100E31009079DDF0907AED04F0E4907AE0F0A3F09F
:100E4100020A599079DF7404F09077BDE02432F5FD
:100E51000A020A599080027410F0750A039079DD34
:100E6100E06401FFF09079DF7401F0EF7019907781
:100E7100B9E06013FCA3E0FDA3E0FEA3E0FF907ADC
:100E8100E91223B5020A599077B5E0FCA3E0FDA36E
:100E9100E0FEA3E0FF907AE91223B5020A5980FE31
:010EA100222E
:100026009077DEE0B444047F0180027F009077DDA4
:10003600E0B447047E0180027E00EE5F604A90775E
:10004600A6E09077DFF09077A7E09077E0F09077E2
:10005600A8E09077E1F09077A9E09077E2F09077CA
:10006600AAE09077E3F09077ABE09077E4F09077B2
:10007600DE7452F090771563A2019080A863A20106
:100086007F06122BA9020877907799E0C39408504F
:10009600030208809077A6E0FF9077DFE06F6003A9
:1000A6000208809077A7E0FF9077E0E06F60030298
:1000B60008809077A8E0FF9077E1E06F6003020880
:1000C600809077A9E0FF9077E2E06F6003020880F6
:1000D6009077AAE0FF9077E3E06F600302088090D4
:1000E60077ABE0FF9077E4E06F60030208809077DB
:1000F600DEE0B44415907715E0B4FF0E63A20190DC
:1001060080A863A2017F06122BA9907AF2E0600311
:100116007401F0907AF37464F09077DE7452F09084
:1001260077DDE0646D60030202A37BFF7A14791A1F
:100136001219A57BFF7A1479349077A6E0F52FA3E0
:10014600E0F530A3E0F531A3E0F532A3E0F533A303
:10015600E0F5341219A5752FFF75301475319175B8
:1001660032FF75331475349D7BFF7A14796A121940
:10017600A57BFF7A1479A61219A57BFF7A15790C4F
:100186001219A57BFF7A1579399077ACE0F52FA384
:10019600E0F530A3E0F531A3E0F5321219A57BFFB7
:1001A6007A1579639077B5E0F52FA3E0F530A3E0F3
:1001B600F531A3E0F5321219A57BFF7A15799190F6
:1001C60077B9E0F52FA3E0F530A3E0F531A3E0F52C
:1001D600321219A57BFF7A1579BF9077A2E0F52F29
:1001E600A3E0F530A3E0F531A3E0F5321219A57BC3
:1001F600FF7A1579E290779EE0F52FA3E0F530A31C
:10020600E0F531A3E0F5321219A57BFF7A1579FFE7
:100216009077BDE0F52F1219A57BFF7A1679291282
:1002260019A57BFF7A167952A20EE433F52F12191F
:10023600A57BFF7A167982907AE8E0F52F1219A548
:100246007BFF7A1679AD907AF2E0F52F1219A57B2D
:10025600FF7A1679E090771BE0F52F1219A57BFF40
:100266007A17790EA201E433F52F1219A57BFF7ACE
:1002760017793A907AE2E0F52FA3E0F530A3E0F59E
:1002860031A3E0F532A3E0F533A3E0F5341219A566
:10029600123BEB7BFF7A1779851219A5229077DD41
:1002A600E0644C70527E177F8B12395C9077E5E0E4
:1002B600F527A3E0F528E4F5297D03AF28AE27123C
:1002C6003A3D7E177FC612395CAE27AF28E4FB7D28
:1002D60010123B177E177FC912395C74102528F55A
:1002E60028E43527F5270529E529C3941040CA7E59
:1002F600177FC912395C229077DDE0646C705CF57B
:100306002B7E177FCB12395CE4F52AAF2B7E007D5E
:1003160003123A3D7E177FC612395CE4F529A82BF5
:10032600E6FF74E72529F582E43477F583EFF005D7
:100336002B0529E529B410E67E777FE7E4FB7D10DF
:10034600123B177E177FC912395C052AE52AC3942A
:100356000840B87E177FC912395C229077DDE064C9
:100366004B7061F52974CF2529F582E43477F5833E
:10037600E0603274CF2529F582E43477F583E0F422
:10038600602374CF2529F582E43477F583E0FF7482
:10039600E52529F582E43477F583E0B507100529CC
:1003A600E529B408C09075697432F0020877907731
:1003B600DD7421F0300A030208777E187F061239B1
:1003C6005C0208779077DDE0B4521A200A077E189F
:1003D6007F0E12395C9077DD7472F07E777FDD7D5B
:1003E600081240BD229077DDE064497045200A0777
:1003F6007E187F1912395C9077E5E0F527A3E0F5C2
:1004060028E4F529852882852783E0FF74E72529D6
:10041600F582E43477F583EFF00528E528700205C8
:10042600270529E529B480DC7E777FDD7D8A1240A9
:10043600BD229077DDE064437079A3E06452704694
:10044600200A077E187F2112395C9077E5E0F527B0
:10045600A3E0F528E4F529852882852783E493FF20
:1004660074E72529F582E43477F583EFF00528E56E
:1004760028700205270529E529B480DB7E777FDD14
:100486007D8A1240BD229077DEE064576003020841
:10049600809077E5E0F527A3E0F52874E72529F5B0
:1004A60082E43477AD82FC7B80AF28AE271246F516
:1004B6000208779077DDE06444600302054A90778E
:1004C600E5E0FF64447003020877EFB4310CC20A1A
:1004D6007E187F2A12395C0208779077E5E0B430FF
:1004E6000CD20A7E187F3612395C0208779077E5BF
:1004F600E0B4320CD20B7E187F4312395C020877C7
:100506009077E5E0B4330CC20B7E187F5112395C4C
:100516000208779077E5E0B4340CD20C7E187F6041
:1005260012395C0208779077E5E0B4350CC20C7E90
:10053600187F6D12395C0208779077E5E0FF1200AC
:100546001E020877907569E07013200A077E187FEF
:100556007B12395C9077DD7421F00208779075691B
:100566007432F09077DDE0FFB4510A908000748019
:10057600F0C2AF80FEEF64577045200A077E187FF1
:100586008912395C9077E6E0907799F0E4F5299046
:100596007799E0FFE529C39F400302087774E725B2
:1005A60029F582E43477F583E0FF9077E5E02529A5
:1005B6002414F582E43476F583EFF0052980D09093
:1005C60077DDE064536003020679200A077E187F10
:1005D6009412395C9077A6E0FF90761DE06F703C30
:1005E6009077A7E0FF90761EE06F70309077A8E0D6
:1005F600FF90761FE0B507249077A9E0FF9076205C
:10060600E0B507189077AAE0FF907621E0B5070CD1
:100616009077ABE0FF907622E06F60169077DD74FE
:1006260021F0300A030208777E187FA312395C0294
:100636000877E4F529E4F50DAF29FE74142529F5AC
:1006460082E43476F583E0FD1248A30529E529C343
:1006560094FE40E19080007480F0C2AFE4907FF099
:10066600F0A3F0907FFD74AAF0A374FFF0A3745575
:10067600F080FE9077DDE0644F704C9077E5E0F512
:1006860027A3E0F528E5284527700A200A077E18E3
:100696007FAC12395C200A077E187FB312395CE4FE
:1006A600F52974E72529F582E43477F583E0852872
:1006B60082852783F00528E528700205270529E5A8
:1006C60029B480DE0208779077DDE0FFB4452790F5
:1006D60080007480F09077E5E0FDA3E0907FF0CD98
:1006E600F0A3EDF0C2AF907FFD74AAF0A374FFF003
:1006F600A37455F080FEEF64656003020877907777
:10070600E5E0FFA3E0907FF0CFF0A3EFF0E4F5275C
:10071600F528D3907FF1E09528907FF0E09527406B
:1007260020E4F50D2528FFE5273401FE852882857E
:100736002783E0FD1248A30528E5287002052780D7
:10074600D17E187FB5123FB4EF4E602012000390A1
:1007560077ACEFF01200039077ADEFF01200039044
:1007660077AEEFF01200039077AFEFF07E187FBB05
:10077600123FB4EF4E60201200039077B5EFF012EF
:1007860000039077B6EFF01200039077B7EFF01200
:1007960000039077B8EFF07E187FC1123FB4EF4E9A
:1007A60060201200039077B9EFF01200039077BA39
:1007B600EFF01200039077BBEFF01200039077BCC6
:1007C600EFF07E187FC7123FB4EF4E602012000391
:1007D6009077A2EFF01200039077A3EFF0120003D8
:1007E6009077A4EFF01200039077A5EFF07E187FC4
:1007F600CD123FB4EF4E602012000390779EEFF0CB
:1008060012000390779FEFF01200039077A0EFF0AD
:100816001200039077A1EFF07E187FD3123FB4EF5A
:100826004E60081245349077BDEFF0E4F529E4F503
:100836000DE5292401FFE433FE749E2529F582E4A3
:100846003477F583E0FD1248A30529E529C39443CF
:1008560040DC9080007480F0C2AFE4907FF0F0A39B
:10086600F0907FFD74AAF0A374FFF0A37455F08096
:0A087600FE7E777FDD7D081240BD95
:010880002255
:1046BD00AE07EEC39430400BEED394395005EE2483
:1046CD00D0FF22EEC39461400BEED394665005EEFD
:1046DD0024A9FF22EEC39441400BEED3944650051E
:0846ED00EE24C9FF22AF0622F2
:10488900907714E004F07006907713E004F09077C5
:0A48990013E0FEA3E0FF12486D22B9
:100003001248891246BDEFC454F0FEC00612488957
:080013001246BDD0E02FFF22D0
:10453400E4907C30F0124889907C31EFF0C39430E1
:104544004018E0FFD394395011907C30E0246CF58E
:1045540082E43475F583EFF08011907C30E0246CB4
:10456400F582E43475F583E4F0800C907C30E0044B
:10457400F0E0D3940840BE752F007530007531000B
:0C458400E4F5327B017A75796C122C8012
:014590002208
:043FB4008E2C8F2D93
:103FB800907713E4F0A374FFF0124889EF606EF471
:103FC800606B852D82852C83E493B507EC752E01F3
:103FD800E52D252EF582E4352CF583E493602590B4
:103FE8007714E0252EFF907713E03400FE12486D19
:103FF800E52D252EF582E4352CF583E493B50704E9
:10400800052E80CCE52D252EF582E4352CF583E4AC
:104018009370A6E52E24FFFFE434FFFE907714E0AA
:104028002FF0907713E03EF07E007F0122E4FEFF40
:014038002265
:103876007E197F04123FB4EF4E70037F01227E193A
:103886007F07123FB4EF4E600C124889EF24D02414
:10389600FF920E8002D20E7E197F0D123FB4EF4EBC
:1038A600600C124889EF24D0907AE8F08005E49005
:1038B6007AE8F07E197F13123FB4EF4E600C12487F
:1038C60089EF24D0907AF2F08005E4907AF2F07EC7
:1038D600197F19123FB4EF4E600C124889EF24D0BD
:1038E60090771BF08005E490771BF07E197F1F12FE
:1038F6003FB4EF4E600C124889EF24D024FF9201AA
:103906008002C2019077A663A201907AE263A201C7
:103916007F06122BA930013B7E197F25123FB4EF9B
:103926004E6030120003907AE2EFF0120003907AB4
:10393600E3EFF0120003907AE4EFF0120003907ABE
:10394600E5EFF0120003907AE6EFF0120003907AAA
:06395600E7EFF07F002204
:10270400C201E4907AF2F0D20EC204907AE8F0901A
:10271400771BF09077A663A201907AE263A2017F0F
:1027240006122BA9E4F527E52775F003A4242BF55D
:1027340082E43419F583E493FB740193FA740293ED
:10274400F912226C70030228F6E4F528F529FD74C9
:10275400942DF582E43475F583E0FF70030228F1CB
:10276400E52775F003A4242BF582E43419F583E4FA
:1027740093FB740193FA740293F98528827583009C
:10278400122285FEEFB5060875290105280228EDF9
:10279400E52970030228EDEE60030228E8E527240A
:1027A400FE60281470030228D01470030228D41485
:1027B40070030228DC1470030228E024056003027D
:1027C40028F1907AF27401F00228F1D20174942D68
:1027D400F582E43475F583E0FF642D70030228F17B
:1027E4001246BDEFC454F0FC74952DF582E43475A3
:1027F400F583E0FF1246BDEF2C907AE2F074962D3B
:10280400F582E43475F583E0FF1246BDEFC454F05D
:10281400FC74972DF582E43475F583E0FF1246BD10
:10282400EF2C907AE3F074982DF582E43475F583F7
:10283400E0FF1246BDEFC454F0FC74992DF582E418
:102844003475F583E0FF1246BDEF2C907AE4F07402
:102854009A2DF582E43475F583E0FF1246BDEFC48A
:1028640054F0FC749B2DF582E43475F583E0FF127B
:1028740046BDEF2C907AE5F0749C2DF582E4347516
:10288400F583E0FF1246BDEFC454F0FC749D2DF5B2
:1028940082E43475F583E0FF1246BDEF2C907AE6AE
:1028A400F0749E2DF582E43475F583E0FF1246BD85
:1028B400EFC454F0FC749F2DF582E43475F583E085
:1028C400FF1246BDEF2C907AE7F08021D204801DE0
:1028D400907AE87401F08015C20E801190771B7411
:1028E40001F08009E4F529F5280D02275305270294
:0228F400272B90
:0128F60022BF
:1045EA009079DEE0C3947C503D9079DEE0FE04F0E1
:1045FA00741C2EF582E43477F583EFF0BF0A279016
:10460A0079DEE0FF04F0741C2FF582E43477F58339
:10461A00E4F09079DEE0FF12413F9079DE7408F011
:07462A0090771DE004F0226F
:104591009080007480F090779E63A201F583F5828C
:1045A10063A2017F08122BA99077A663A2019080D4
:1045B1008863A2017F0A122BA9908092E4F0A37470
:1045C10032F0A37401F09077B0E0FF9080B1F090E9
:1045D10080E1EFF09080957455F0A3F09080007425
:0945E10001F09080097470F022D1
:1042B600908009E04410F09080A0E0706C9080A19E
:1042C6007482F09080A874FFF0A3F0A3F0A3F07FAF
:1042D600039080AEEFF07FCBA3EFF07F039080AC2E
:1042E600EFF0A374CBF09080007402F0907C221261
:1042F60023C100000000907C22E0908040F0907C7A
:1043060023E0908041F0907C24E0908042F0907C05
:1043160025E0908043F0A3E4F0A3F0A3F0A3F0908F
:094326008018F0A3F0A3F0A3F04D
:01432F00226B
:10440F00908009E04440F09080D17482F09077B1B1
:10441F00E0FF9080DEF09077B2E0FF9080DFF090C9
:10442F0080027402F0907C261223C10000000090DD
:10443F007C26E0908058F0907C27E0908059F09097
:10444F007C28E090805AF0907C29E090805BF0A36C
:10445F00E4F0A3F0A3F0A3F0908030F0A3F0A3F06A
:02446F00A3F0B8
:014471002228
:10433000908009E04420F09080B8E0706C9080B9E3
:104340007482F07F039080C6EFF07FCDA3EFF07F03
:10435000039080C4EFF0A374CDF09080C074FFF0A0
:10436000A3F0A3F0A3F09080017402F0907C2A12D5
:1043700023C100000000907C26E090804CF0907CEF
:1043800027E090804DF0907C28E090804EF0907C6B
:1043900029E090804FF0A3E4F0A3F0A3F0A3F09005
:0943A0008024F0A3F0A3F0A3F0C7
:0143A90022F1
:104039008C278D28A907EAFDE975F018A424ACFF9F
:10404900E5F034808F82F583EDF0EBFDE975F0182A
:10405900A4FFAEF024ACFBEE34808B82F583A3ED94
:10406900F08528828C83E0FDEF24A8FFEE3480FEE2
:104079008F82F583EDF08528828C83A3E08F828E71
:1040890083A3F0852882852783A3A3E0FDE975F042
:1040990018A424A8FFE5F03480FE8F82F583A3A33A
:1040A900EDF08528828C83A3A3A3E08F828E83A35E
:0440B900A3A3F022AB
:0640BD008D2CAB07AA06E2
:1040C300907C22E0FCA3E0FDA3E0FEA3E0F5308EAC
:1040D3002F8D2E8C2DAE02AF038E838F8263A201B0
:1040E300E52F540744C0F58385308263A201AF2CCA
:1040F300122C12908000E020E5F9E4FCFDFEE5308F
:10410300252CF530EE352FF52FED352EF52EEC352C
:104113002DF52D908040E52DF0A3E52EF0A3E52F9E
:10412300F0A3E530F09080007420F0AF30AE2FADF7
:0B4133002EAC2D907C221223B5AF2C87
:01413E00225E
:06423B008D27AB07AA0667
:10424100907C26E0FCA3E0FDA3E0FEA3E0F52B8E2D
:104251002A8D298C28AE02AF038E838F8263A2013F
:10426100E52A540744D0F583852B8263A201AF2749
:10427100122C12E4FCFDFEE52B2527F52BEE352A49
:10428100F52AED3529F529EC3528F528908058E5F2
:1042910028F0A3E529F0A3E52AF0A3E52BF090800F
:1042A100027420F0AF2BAE2AAD29AC28907C2612E7
:0442B10023B5AF275B
:0142B50022E6
:023CBF008F284C
:103CC100908001E030E5037F0022907C2AE0FCA394
:103CD100E0FDA3E0FEA3E0F52C8E2B8D2A8C29902C
:103CE1007AE263A201E52B540744C8F583852C824F
:103CF10063A2017F06122C28E52C2406F52CE4355D
:103D01002BF52BE4352AF52AE43529F5299079E0BC
:103D110063A201E52B540744C8F583852C8263A275
:103D210001AF28122C28E4FCFDFEE52C2528F52CFA
:103D3100EE352BF52BED352AF52AEC3529F52990B1
:103D4100804CE529F0A3E52AF0A3E52BF0A3E52CAF
:103D5100F09080017420F0AF2CAE2BAD2AAC2990ED
:073D61007C2A1223B5AF28F4
:013D68002238
:103772009081E0E0F527052705270527052705277E
:1037820005270527052705270527908010E0F52A3C
:10379200A3E0F52BA3E0F52CA3E0F52D9081E1E069
:1037A200F5270527052705270527052705270527C7
:1037B200052705270527908014E0F52EA3E0F52FB5
:1037C200A3E0F530A3E0F531E530B52C08E531B5DD
:1037D2002D037F0022E4F527E530540744E0F5830A
:1037E20085318263A2019077DD63A2017F08122CEA
:1037F200409077DF63A20190771563A2017F0612E2
:103802002BA99077DDE0F528A3E0F529E4F52790D0
:1038120077DDE0702AA3E024F8F527E53054074469
:10382200E0F58385318274082582F582E43583F5DB
:103832008363A2019077DD63A201AF27122C40AE11
:1038420028E4FCFDE5312529F531E5303EF530ED82
:10385200352FF52FEC352EF52E908014E52EF0A3A2
:10386200E52FF0A3E530F0A3E531F090800074403D
:03387200F0AF278D
:013875002230
:102FC2009081E6E0F5270527052705270527052730
:102FD20005270527052705270527908028E0F52ADC
:102FE200A3E0F52BA3E0F52CA3E0F52D9081E7E01B
:102FF200F52705270527052705270527052705277F
:1030020005270527052790802CE0F52EA3E0F52F54
:10301200A3E0F530A3E0F531E4F527E530B52C0A5D
:10302200E531B52D05C20802311CE530540744F0E4
:10303200F58385318263A2019077DD63A2017F0867
:10304200122C409077DDE0F528A3E0F529E529452B
:103052002870099080027410F07F0022907AE9E0D3
:10306200FFF4602D9077DFE06F7076907AEAE0FFF0
:103072009077E0E06F706A907AEBE0FF9077E1E0A2
:103082006F705E907AECE0FF9077E2E06F602280F2
:10309200509077DFE0907AE9F09077E0E0907AEA7A
:1030A200F09077E1E0907AEBF09077E2E0907AECC2
:1030B200F09077DDE0702AA3E024F8F527E530549C
:1030C2000744F0F58385318274082582F582E43560
:1030D20083F58363A2019077DD63A201AF27122CEF
:1030E20040AE28E4FCFDE5312529F531E5303EF519
:1030F20030ED352FF52FEC352EF52EAF2DAE2CAD54
:103102002BAC2AAB31AA30A92FA82ED31223A4406C
:10311200099080027410F07F002290802CE52EF03E
:10312200A3E52FF0A3E530F0A3E531F0908002741F
:0431320040F0AF2793
:013136002276
:103137009081E3E0F52705270527052705270527BC
:103147000527052705270527052790801CE0F52A71
:10315700A3E0F52BA3E0F52CA3E0F52D9081E4E0A7
:10316700F527052705270527052705270527052708
:10317700052705270527908020E0F52EA3E0F52FEA
:10318700A3E0F530A3E0F531E4F527E530B52C0AE7
:10319700E531B52D05C209023282E530540744E80E
:1031A700F58385318263A20190746963A2017F0E62
:1031B700122C56907469E0F528A3E0F529907471F4
:1031C700E0FFF46045907AE2E0FEEF6E706EA3E0F8
:1031D700FF907472E06F7064907AE4E0FF9074730C
:1031E700E06F7058907AE5E0FF907474E06F704C70
:1031F700907AE6E0FF907475E06F7040907AE7E0B0
:10320700FF907476E06F60048032D2D9907469E0E1
:10321700702AA3E024F2F527E530540744E8F58344
:10322700853182740E2582F582E43583F58363A2A6
:103237000190746963A201AF27122C56AE28E4FCF3
:10324700FDE5312529F531E5303EF530ED352FF532
:103257002FEC352EF52EAF2DAE2CAD2BAC2AAB3186
:10326700AA30A92FA82ED31223A45006E529452852
:1032770070099080017410F07F0022908020E52E65
:10328700F0A3E52FF0A3E530F0A3E531F09080013E
:053297007440F0AF27B8
:01329C00220F
:04395C008E2C8F2DF1
:10396000907C22E0FCA3E0FDA3E0FEA3E0F5338E13
:10397000328D318C30E533FFE5325407FEE42FF50C
:103980002FEE34C0F52E852F82F5837423F0052F9A
:10399000E52F7002052E532EC7F582852E83740AFB
:1039A000F0052FE52F7002052E532EC79077A663E2
:1039B000A201852E83852F8263A2017F06122C121D
:1039C0007406252FF52FE4352EF52E852C83852DB5
:1039D0008263A201852E83852F8263A201122BF6BA
:1039E000908000E020E5F9E4FCFDFE907C22E0F808
:1039F000A3E0F9A3E0FAA3E02FFFEE3AFEED39FDD4
:103A0000EC38FCEF2408FFE43EFEE43DFDE43CFC22
:103A1000907C221223B5907C22E0908040F0907C34
:103A200023E0908041F0907C24E0908042F0907CF4
:0C3A300025E0908043F09080007420F0AE
:013A3C002267
:063B17008E2C8F2D8D2E77
:103B1D00907C22E0FCA3E0FDA3E0FEA3E0F5348E53
:103B2D00338D328C31E534FFE5335407FEE42FF548
:103B3D0030EE34C0F52F853082F5837423F00530D7
:103B4D00E5307002052F532FC7F582852F83EBF0DB
:103B5D000530E5307002052F532FC79077A663A26D
:103B6D0001852F8385308263A2017F06122C12748A
:103B7D00062530F530E4352FF52F852C83852D82E4
:103B8D0063A201852F8385308263A201AF2E122C93
:103B9D0012908000E020E5F97408252EF52EFFE443
:103BAD00FCFDFEE5342FF534EE3533F533ED3532CE
:103BBD00F532EC3531F531908040E531F0A3E53249
:103BCD00F0A3E533F0A3E534F09080007420F0AF5E
:0D3BDD0034AE33AD32AC31907C221223B5F2
:013BEA0022B8
:02413F008F40AF
:10414100907C22E0FCA3E0FDA3E0FEA3E0F5448E19
:10415100438D428C41E544FFE5435407FEE42FFFC4
:10416100EE34C090771C63A201F5838F8263A201B4
:10417100AF40122C12908000E020E5F9E4FCFDFE36
:10418100E5442540F544EE3543F543ED3542F5422E
:10419100EC3541F541908040E541F0A3E542F0A3C3
:1041A100E543F0A3E544F09080007420F0AF44AE05
:0B41B10043AD42AC41907C221223B5CC
:0141BC0022E0
:063A3D008E2C8F2DAB055D
:103A4300907C22E0FCA3E0FDA3E0FEA3E0F5338E2F
:103A5300328D318C30E533FFE5325407FEE42FF528
:103A63002FEE34C0F52E852F82F5837423F0052FB6
:103A7300E52F7002052E532EC7F582852E83EBF0BA
:103A8300052FE52F7002052E9077A663A201852EE0
:103A930083852F8263A2017F06122C127406252FC1
:103AA300F52FE4352EF52E532EC7E52C852F828571
:103AB3002E83F0052FE52F7002052E532EC7F582B6
:103AC300852E83E52DF0052FE52F7002052E532E4D
:103AD300C7908000E020E5F9E533240AF533E435A7
:103AE30032F532E43531F531E43530F5309080404C
:103AF300E530F0A3E531F0A3E532F0A3E533F09030
:103B030080007420F0AF33AE32AD31AC30907C2204
:033B13001223B5C5
:013B1600228C
:10486D00E5D220E0FBC2AF438E2075D2028F828E3F
:0B487D0083E0FFE4F5D2538EDFD2AFE2
:01488800220D
:1048A300E5D220E0FBC2AF43D2028F828E83EDF0CC
:0948B30075D25063D250D2AF223D
:1041BD00E4FDED2401FFE433FE12486D749E2DF5F0
:1041CD0082E43477F583EFF00DBD3FE6E4FDED2499
:1041DD007FFFE433FE12486D74942DF582E434753F
:1041ED00F583EFF074942DF582E43475F583E0706A
:1041FD001B74942DF582E43475F5837420F0749559
:10420D002DF582E43475F583E4F080040DBD80BE98
:10421D00E4907613F0FDEDFF7E0012486D74142DC1
:0D422D00F582E43476F583EFF00DBDFEE977
:01423A002261
:0246F5008B2C0C
:1046F700A2AF921DC2AF85A22D53A2FE8E838F82D9
:1047070005A28C838D827409122C6EE52C53A2FEB0
:1047170043A220122C7053A2DF852DA2A21D92AFB7
:01472700FF92
:01472800226E
:10485000A2AF921DC2AF8C838D82EF122C6E43A249
:0C48600020122C7053A2DFA21D92AFFFAB
:01486C002229
:024808008F27F8
:10480A00A2AF921DC2AFE4F5838D827406122C6E9C
:10481A00E52743A220122C7053A2DFA21D92AF7F7C
:01482A00018C
:01482B00226A
:02482C008F27D4
:10482E00A2AF921DC2AFE4F5838D82740A122C6E74
:10483E00E52743A220122C7053A2DFA21D92AF7F58
:01484E000168
:01484F002246
:102ACE00A907E7FFA805EF93C3966008403B74FC87
:102ADE002FFF80F00F08EF93C3966008402B74FB16
:102AEE002FFF80E00F08EF93C3966008401B74FA27
:102AFE002FFF80D00F08EF93D3966008400B74F928
:102B0E002FFF80C01F1F1F1F1FEF54FEF80303F778
:102B1E00E893FC08E893FD08E893FE08E893FF228B
:102B2E0009E993C39D6008402974FB29F980F109D6
:102B3E00E993C39E6008401A74FA29F980E209E904
:102B4E0093D39F6008400B74F929F980D319191992
:102B5E001919E9C313C313FF22740093F8ECC39839
:102B6E004024701F740193F8EDC3984019701474CB
:0E2B7E000293F8EEC398400E7009740393F8AA
:102B8C00EFC39840037F00227F0122EDF8E6F008A6
:102B9C00A3DFFA22EDF8E0F608A3DFFA22E0A36344
:102BAC00A201F0A363A201DFF475A20022E0A363EB
:102BBC00A201F0A363A201E0A363A201F0A363A2AC
:102BCC0001E463A201F0A363A201DFE175A200227C
:102BDC00E0A363A2016DFE936CFDEE058393FC15DF
:102BEC008363A201DFEA75A200227F00E493A36352
:102BFC00A201F00F600CA3E583C2E3F58363A2018D
:102C0C0080EA75A20022E0A363A201F0A3E583C2CF
:102C1C00E3F58363A201DFEE75A20022E0A363A2B9
:102C2C0001F0A3E583C2E4D2E3F58363A201DFECF8
:102C3C0075A20022E583C2E3F583E0A363A201F051
:102C4C00A363A201DFEE75A20022E583C2E4D2E306
:102C5C00F583E0A363A201F0A363A201DFEC75A2EC
:102C6C000022F922C002C004C00612FFF0D006D028
:042C7C0004D002225C
:103E9A000A536572763A004572724C656E210A00C1
:103EAA00205544502054696D654750530A00200A32
:103EBA00444154414752414D3A20002043414E204B
:103ECA0054696D654750530A0020547261737353E5
:103EDA00656E644552520A000ACEF8C4EBE8EDFB5F
:103EEA0043414E210A000A45727241647243414EAF
:103EFA003A000A00205265496E69742043414E0A0D
:103F0A00002043414E283029203E20544F210A00E8
:0E3F1A0020545520300A0020545520310A0052
:03001E00E4FF22DA
:1047B900C2A9438902758C48758A4875D90475DB85
:1047C9004875DC4875DD4875DE48E4F5E9F5F9D248
:0847D900D9C2DAD28CD2DE2233
:10478B00C2D9907B08E07013E5E92419F5EB30D71B
:10479B0006E5F904F5FB2285F9FB22E5E924C8F5CA
:0E47AB00EB30D706E5F904F5FB2285F9FB2279
:10463100C2D9907B08E0702C302A16E5E92432F5C6
:10464100EB30D707E5F904F5FB800385F9FBC22AB6
:1046510022E5E92405F5EB30D706E5F904F5FB225F
:1046610085F9FB22E5E92432F5EB30D706E5F904BB
:07467100F5FB2285F9FB2295
:1047E1001247B9907B08E0C3946450061243AA12A1
:1047F100478B120022D229E4F556907C20F0F54532
:07480100F55AC22AF5582206
:10467800EF24FCF545200A127E3E7F9A12395C7EB3
:10468800777FE1E4FBAD45123B17E545D3940D4038
:1046980010200A077E3E7FA112395CE4F545D22737
:1046A800229077E163A201907C1063A201AF4512CA
:0546B8002BA9C227221E
:0F48D000D3EF6480948D5006E55A70028F5A2200
:101F990020D903022076202903022076E55A6052CF
:101FA900907469540FFF7D47122BA0E547640170B7
:101FB9001E907471E0B4FF0ED22B200A127E3E7F70
:101FC900AA12395C8009302B06E4F55A02207612F0
:101FD900478B124472200A077E3E7FB812395C2073
:101FE9000A0B7E747F69E4FBAD5A123B17E4F55A7C
:101FF900807BE5456043907C14E02405F527D39464
:102009000D4007E4F545D2278063907C10E52754FD
:102019000FFF7D47122BA0E54730E702D22AE5479B
:10202900B40109302B06E54A6401600312447212B7
:10203900478BE4F545D2278034E557601E907AF442
:10204900540FFF7D47122BA0E547B40103202B0352
:1020590012447212478BE4F5578012200F0C907BC3
:1020690008E0C3946450031244D412478B12329D82
:102079008F27EF700302213D124631E4F558E547F9
:10208900B4010CD22B200A077E3E7FC512395CE5CC
:1020990059C394C8502D30032AE547B4420DE54A87
:1020A900B4020890771BE06401601874092559F59A
:1020B90082E4347BF583E5272559F5597D47AF2718
:1020C900122B97300121E54720E71C9079E07D47E5
:1020D900AF27122B97AF27123CBFEF700A200A07D0
:1020E9007E3E7FD312395CE54754817047E527D39B
:1020F900940D400C200A3D7E3E7FE212395C80340B
:10210900E549D394074028200A2A7E3E7FF01239F8
:102119005C90756C7D47AF27122B977E757F6CE4B9
:10212900FBAD27123B177E3E7FFC12395C8005AF61
:10213900271233F5300D2030001B907B08E0C39443
:102149006450120558E55894F0400A908000748054
:10215900F0C2AF80FEC20D20020302226690600128
:10216900E004F07006906000E004F0E5566031D3B9
:102179009401400415568028907C20E004F0E0D3B7
:102189009403400D200A077E3E7FFE12395C1247F8
:10219900E1200A077E3F7F0B12395CE4F556D2290C
:1021A900302843E557703F907AF404F0A37408F09F
:1021B900A37480F0A37401F0A37406F0907C0BE083
:1021C900907AF9F0907C0CE0907AFAF0907C0DE02E
:1021D900907AFBF0907C0EE0907AFCF0E4A3F0A3F7
:1021E900F075570BC228302672907C09E07035E5EE
:1021F900577031907AF47442F0A37408F0907C0A15
:10220900E0907AF6F0907C0FE0907AF7F0A37401F1
:10221900F0755706200A077E3F7F1A12395C907CB9
:1022290009E004F0907C09E06402702FE557702BF7
:10223900907AF47402F0A37408F0907C0AE0907A22
:10224900F6F0A3F0A37401F0755706200A077E3F44
:102259007F2112395C907C09E004F0C202122E241D
:02226900C200B1
:01226B002250
:10472900E559602CE49078DDF0A3E559F0907AE141
:10473900E09078DFF0A37419F0907B0963A20190EF
:1047490078E163A201AF59122BA9E4F5597F01223F
:034759007F0022BC
:0B48DF00302705C2277F01227F002246
:0100210022BC
:06490400E4F559F545221F
:0A48EA00E490756CF0A3F0A3F02237
:10475C002043616E457247495400200A004572722D
:10476C004C656E43616E21000A002043616E4572F8
:0F477C0072434821000A20526571457272210074
:10329D00E59B541F6020200A1A7E477F5C12395C23
:1032AD00E59B541FFF7E007D03123A3D7E477F66EE
:1032BD0012395CE4F59BE5BA30E010E4F5B375B175
:1032CD0080F5B2D229F556907C20F0E5CFF470034D
:1032DD000233F2752901E4F528E5CFF45529700381
:1032ED000233E0E528C454F0F5B1E5B2547F642013
:1032FD0060030233B1E5B3540FF54B85BC47E5BD13
:10330D00541FFF131313541FFFE5BD54E044184F12
:10331D00F548E5BDC43354E0FFE5BE131313541F48
:10332D004FF549E5BEC43354E0FFE5BF1313135405
:10333D001F4FF54A85A34C85A34D85A34E85A34FFD
:10334D0085A35085A35185A35285A353E4F5B220DF
:10335D000F0CE547547EB5470575B350800375B323
:10336D00D0E54B700AE547547EB547037F00223008
:10337D000F08E54730E7037F0022E54BD394084063
:10338D001D200A177E477F6912395CAF4B7E007D89
:10339D0003123A3D7E477F7412395C7F0022E54B64
:1033AD002405FF22E5B2549F6023200A207E477F2B
:1033BD007612395CAFB27E007D03123A3DAFB37E1B
:1033CD00007D03123A3D7E477F7412395CE4F5B2FD
:1033DD0075B3D0E52925E0F5290528E528C394081E
:0733ED0050030232E67F00ED
:0133F40022B6
:10447200907B08E0C39464505675B180E4F5B3F5BF
:10448200B28547BCE549C4135407FFE54854E04FE1
:10449200F5BDE54933333354F8FFE54AC4135407F5
:1044A2004FF5BEE54A33333354F8F5BF854CA38547
:1044B2004DA3854EA3854FA38550A38551A3855255
:1044C200A38553A3E54B540F2450F5B375560AC286
:0244D20029229D
:1044D40075B190E5B220E613200A107E477F811261
:1044E400395CAFB27E007D03123A3DE4F5B3F5B218
:1044F4007472250FF582E43461F583E0F5BCE4F5CC
:10450400BD7473250FF582E43461F583E0FF333322
:104514003354F8F5BE75BF78050F050F7472250F77
:10452400F582E43461F583E07002F50F75B350222F
:0948F400EF6003C29622D2962265
:1043AA0043AB01C2E8C2EAE4FFEFC454F0F5B1C37B
:1043BA00EF64809488500575B3D08003E4F5B3E4C4
:1043CA00F5B2F5BCF5BDF5BEF5BFF5C4F5C5F5C644
:1043DA00F5C7F5A3F5A3F5A3F5A3F5A3F5A3F5A3EF
:1043EA00F5A30FBF0EC3907B08E0FF25E0F5B47577
:1043FA00B50C75B66C75A11275AB0275C13E75C365
:04440A00FF75C20375
:01440E00228B
:100EA2005452414E5A004D4158420052545300444C
:100EB200454C4159004E4F4B5654004B5000424F47
:100EC2004F540043414E004E4557504B540041543D
:100ED200004443440043414E4D4F4E0054454C3A6A
:100EE200004C434C004454420054524300003E2AFA
:100EF2002C312CCFE0F0E0ECE5F2F0FB20F3EFF048
:100F0200E0E2EBFFFEF9E5E3EE20EAEEEDF2F0EED1
:100F1200EBEBE5F0E020CACF20C8F1E5F2FC0A00D5
:100F22003E4C2C6B30312C25732C43EAEEF0EEF163
:100F3200F2FC20EDE020F8E8EDE52043414E2C30B4
:100F4200202D20353030EAE1283530EC292C3120B3
:100F52002D203530EAE128353030EC290A003020E6
:100F62002D20353030EAE1283530EC290031202DB2
:100F7200203530EAE128353030EC29003E532C6B25
:100F820030322C2562752CCCE0EAF12E20E0E4F020
:100F9200E5F120E1EBEEEAE020D2D128302D38292C
:100FA2000A003E532C6B30332C2562752CCCE0EAC0
:100FB200F12E20E0E4F0E5F120E1EBEEEAE020D2D0
:100FC200C8D228302D38290A003E532C6B30342CDD
:100FD2002562752CCCE0EAF12E20E0E4F0E5F12068
:100FE200E1EBEEEAE020D2D328302D38290A003E88
:100FF200422C6330312C2562752CC2F2EEF0E8F7F8
:10100200EDFBE920EAEEEDF2F0EEEBEBE5F020EDA0
:10101200E020F8E8EDE50A003E2A2C312CCFE0F082
:10102200E0ECE5F2F0FB20EFF0EEF2EEEAEEEBE0C0
:1010320020C8F1E5F2FC20EFEE20EFEEF0F2F32013
:1010420052533233320A003E4C2C6B30352C256C15
:10105200752CD1EAEEF0EEF1F2FC20EEE1ECE5EDDA
:10106200E020EDE020EFEEF0F2F32C3130302C32C4
:1010720030302C3330302C3630302C313230302C72
:10108200323430302C343830302C393630302C3148
:10109200393230302C33383430302C35373630302A
:1010A2002C3131353230300A003E532C6B30362C25
:1010B2002562752CCAEEEB2DE2EE20E1EBEEEAEEB4
:1010C200E220E220EFE0EAE5F2E50A003E422C6B84
:1010D20030392C2562752CCDE520EFE5F0E5E4E012
:1010E200E2E0F2FC20E4E8E0E3EDEEF1F2E8EAF31C
:1010F2000A003E422C6B31302C2562752CD0E5F172
:10110200F2E0F0F220EFF0E820EEF2F1F3F2F1F289
:10111200E2E8E820EFE5F0E5E4E0F7E820EFE0EAD6
:10112200E5F2EEE2203220ECE8ED2E0A003C21004E
:101132003C6B30313D003C6B30323D003C6B303318
:101142003D003C6B30343D003C6330313D003C6B34
:1011520030353D003C6B30363D003C6B30393D0054
:101162003C6B31303D0043796354530A004D657343
:10117200730A00435449490A00435449540A00532C
:10118200705449540A0054696D655449540A000A5E
:101192004173796E634F55543A00CEF820E4EBE880
:1011A200EDFB210A000A435243204552523A2000E5
:1011B2000A494E3A000A4173796E63494E3A003F3A
:1011C2003F3F0A000089129B24AD36BF48C15AD363
:1011D2006CE57EF78108931AA52CB73EC940DB5215
:1011E200ED64FF76028B109926AF34BD4AC358D105
:1011F2006EE77CF5830A9118A72EB53CCB42D950F5
:10120200EF66FD74048D169F20A932BB4CC55ED7D4
:1012120068E17AF3850C971EA128B33ACD44DF56D4
:10122200E960FB72068F149D22AB30B94EC75CD5C4
:101232006AE378F1870E951CA32AB138CF46DD54B4
:10124200EB62F97008811A932CA53EB740C952DBB4
:1012520064ED76FF89009B12AD24BF36C148D35A94
:10126200E56CF77E0A8318912EA73CB542CB50D984
:1012720066EF74FD8B029910AF26BD34C34AD15874
:10128200E76EF57C0C851E9728A13AB344CD56DF54
:1012920060E972FB8D049F16A920BB32C54CD75E54
:1012A200E168F37A0E871C952AA338B146CF54DD44
:1012B20062EB70F98F069D14AB22B930C74ED55C34
:1012C200E36AF17800112332465765748C9DAFBEF4
:1012D200CADBE9F810013322564775649C8DBFAE14
:1012E200DACBF9E82130021367764455ADBC8E9F04
:1012F200EBFAC8D93120120377665445BDAC9E8FF4
:10130200FBEAD8C94253617004152736CEDFEDFCE3
:101312008899ABBA5243716014053726DECFFDECD3
:101322009889BBAA6372405125340617EFFECCDDC3
:10133200A9B88A9B7362504135241607FFEEDCCDB3
:10134200B9A89A8B8495A7B6C2D3E1F008192B3AB3
:101352004E5F6D7C9485B7A6D2C3F1E018093B2A93
:101362005E4F7D6CA5B48697E3F2C0D129380A1B83
:101372006F7E4C5DB5A49687F3E2D0C139281A0B73
:101382007F6E5C4DC6D7E5F48091A3B24A5B697863
:101392000C1D2F3ED6C7F5E49081B3A25A4B796853
:1013A2001C0D3F2EE7F6C4D5A1B082936B7A485943
:1013B2002D3C0E1FF7E6D4C5B1A092837B6A584933
:1013C2003D2C1E0FFF0EA2FF0EA8FF0EADFF0EB1A9
:1013D200FF0EB7FF0EBDFF0EC0FF0EC5FF0EC9FF09
:1013E2000ED0FF0ED3FF0ED7FF0EDEFF0EE3FF0E71
:0713F200E7FF0EEBFF0EEF19
:030023000235495A
:0B354900C0E0C083C082C0D075D01865
:1035540030984EC298750B01AF9920100FEF64029A
:10356400703F90616CF0D210D2918035301707C251
:1035740017531F0F801CBF0904D2178024BF0312E6
:1035840085616C636180536180C210750B00C291C8
:10359400800F74222561F582E4346FF583EFF00522
:1035A40061209903023662201103023660301673DB
:1035B400E568B4FF0D7599020568756D00D2900237
:1035C4003660E568B560147599030568906F1FE06F
:1035D40070030236607401F0023660E568D39560CA
:1035E4004008C211D21CC2908072E56D6009F59941
:1035F4000568756D00806574222568F582E4347071
:10360400F583E0F56D6402600BE56D64036005E528
:103614006DB409057599098043856D990568756DC3
:1036240000803974222568F582E43470F583E0FF64
:103634007008C211D21CC2908022D290C21CEFB476
:103644007C090568750832C2118011AF6805687479
:0E365400222FF582E43470F583E0F599C299D7
:09366200D0D0D082D083D0E03238
:103BEB007BFF7A0E79F01219A5907B08E0701475A3
:103BFB002FFF75300F7531607BFF7A0F7922121909
:103C0B00A58012752FFF75300F75316F7BFF7A0F03
:103C1B0079221219A57BFF7A0F797E906171E0F5FD
:103C2B002F1219A57BFF7A0F79A490616BE0F52F0A
:103C3B001219A57BFF7A0F79CB906102E0F52F1259
:103C4B0019A57BFF7A0F79F1A20FE433F52F121927
:103C5B00A57BFF7A10791A1219A5907463E0FEA365
:103C6B00E0FFC3E49FFFE49EFEAB07FAE4F9F8FF25
:103C7B007E8C7D0AFC1223048F328E318D308C2F7B
:103C8B007BFF7A1079491219A57BFF7A1079AB85E6
:103C9B00692F1219A57BFF7A1079CEA218E433F5A0
:103CAB002F1219A57BFF7A1079F4906F1FE0F52F77
:043CBB001219A52213
:10366B007E117F2F123FB4EF4E70037F0122E49047
:10367B007B08F07E117F32123FB4EF4E601512487B
:10368B0089BF3106907B08740AF0BF3206907B0825
:10369B007464F07E117F38123FB4EF4E6008124510
:1036AB0034906171EFF07E117F3E123FB4EF4E60AC
:1036BB000812453490616BEFF07E117F44123FB4DA
:1036CB00EF4E6008124534906102EFF07E117F4A95
:1036DB00123FB4EF4E600D124534EC4D4E4F24FFAC
:1036EB00920F8002C20F7E117F50123FB4EF4E60DB
:1036FB0023124534A804A905AA06AB077F007E8CCC
:10370B007D0A7C00122304122396907463EEF0A3BF
:10371B00EFF0800A90746374FFF0A374DCF07E11F9
:10372B007F56123FB4EF4E60071245348F6980030A
:10373B00756902E56970037569017E117F5C123F43
:10374B00B4EF4E600A124889EF24D024FF92187E02
:10375B00117F62123FB4EF4E600A124889EF24D0FA
:06376B00906F1FF07F00CB
:013771002235
:1028F700E4F50F907C30F0907C30E075F003A42471
:10290700C6F582E43413F583E493FB740193FA74F8
:102917000293F912226C7003022ACDE4907C32F004
:10292700A3F0907C31F0907C31E02494F582E4347C
:1029370075F583E0FF7003022AC4907C30E075F0E0
:1029470003A424C6F582E43413F583E493FB7401EE
:1029570093FA740293F9907C32E0F5827583001242
:102967002285FEEFB5060F907C337401F0907C3220
:10297700E004F0022ABB907C33E07003022ABBEE2E
:102987006003022AB2907C30E014607424FC700368
:10299700022A74147003022AA2147003022A442420
:1029A700F97003022AA6147003022AAA240F6003EF
:1029B700022AC4907C31E02494F9E43475FA7B014F
:1029C700C0031B8B2F753000753100E4F532D0033F
:1029D700122C80907C341223B5907C34E0F8A3E06D
:1029E700F9A3E0FAA3E0FB7F007E8C7D0A7C00124E
:1029F7002304122396907463EEF0A3EFF0022AC427
:102A0700907C31E0FD2494F582E43475F583E0246D
:102A1700D0906171F074952DF582E43475F583E0FB
:102A270024D090616BF0907C31E02496F582E434F9
:102A370075F583E024D0906102F0022AC4907C31BE
:102A4700E02494F9E43475FA7B01C0031B8B2F75DE
:102A57003000753100E4F532D003122C80907C34BD
:102A67001223B5907C37E0907B08F08050907C3142
:102A7700E02494F9E43475FA7B01C0031B8B2F75AE
:102A87003000753100E4F532D003122C80907C348D
:102A97001223B5907C37E0F56B8022D212801ED2CC
:102AA70018801A906F1F7401F08012E4907C33F045
:102AB700907C32F0907C31E004F002292D907C303C
:062AC700E004F00228FE0D
:012ACD0022E6
:1024FF00E4906170F09061B5F0C21590616EF0904C
:10250F006F1E7405F0C211C21CC210C217E4F56829
:10251F00F560F508F561F50B90746374FFF0A37423
:10252F00F4F09061027402F090616BF0906171F0C1
:10253F00C21AD219C20F907122741EF0E4907B0858
:10254F00F0C212C214C213F56BC218906F1FF0D2F3
:10255F001612366BEF60031228F7907122E0049089
:10256F00616DF0E4F50F907C2E7461F0A37472F03E
:10257F00906171E0F50FE50FC394014007E50FD3AC
:10258F0094084003E4F50FE50F6028907C2EE47566
:10259F00F0011222B285F082F58374C4F0150F900A
:1025AF007C2EE475F0011222B285F082F583E50FDF
:1025BF00F080D490616BE0F50FE50FC394014007F5
:1025CF00E50FD394084003E4F50FE50F6028907CE6
:1025DF002EE475F0011222B285F082F58374C8F0F3
:1025EF00150F907C2EE475F0011222B285F082F562
:1025FF0083E50FF080D4906102E0F50FE50FC394EF
:10260F00014007E50FD394084003E4F50FE50F6091
:10261F0028907C2EE475F0011222B285F082F583AA
:10262F0074C2F0150F907C2EE475F0011222B28562
:10263F00F082F583E50FF080D4907C2EE475F001E5
:10264F001222B285F082F583E4F0907C2E75F001B2
:10265F001222B285F082F583E4F0F50FF56A75F07A
:10266F0075E56AA42436F582E5F03468F583E4F065
:10267F00E56A75F00DA42403F582E43461F583E473
:10268F00F0F55F75F068E56AA42423F582E5F03470
:10269F0071F58375F00DE55F1223F2E4F0055FE548
:1026AF005FB408DF056AE56AB408B3E4F56FF55B5C
:1026BF00F55DF55EF567F56EF55FF55CF56AF56648
:1026CF00C2ADF5C9D2CDD2CCC2C9C2CAF5CDF5CCF7
:1026DF00907463E0F5CBA3E0F5CA85CBCD85CACC6A
:1026EF00D29ED29CD2CAC2ACC298C29975B810758C
:0426FF00B710D2AC92
:0127030022B3
:0100220022BB
:1033F5008F2830180EE547B44209E54A6402700388
:10340500023548E54854E324DF606D24DF6042144B
:10341500603F24E370030234A41470030234F614ED
:10342500700302352724E2602824606003023548D2
:10343500300B077E117F6812395CE54975F00DA4E4
:103445002403F582E43461F5837D47AF28122B9779
:1034550022300B077E117F6F12395C75F00DE55E2A
:10346500A424DEF582E5F0346BF5837D47AF2812A1
:103475002B97055E535E3F22300B077E117F751239
:10348500395C75F00DE55BA424B6F582E5F0346191
:10349500F5837D47AF28122B97055B535B7F223061
:1034A5000B077E117F7B12395C75F075E549A42405
:1034B50043F582E5F03468F583E54A541FFF13139D
:1034C500543F75F00D1223F27D47AF28122B9775E7
:1034D500F068E549A42423F582E5F03471F583E528
:1034E5004A541FFF1313543F75F00D1223F2E4F0F5
:1034F50022300B077E117F8112395C75F068E54932
:10350500A42423F582E5F03471F583E54A543FFFA1
:103515001313543F75F00D1223F27D477F0D122BC7
:103525009722300B077E117F8812395C75F075E59F
:1035350049A42436F582E5F03468F5837D47AF2844
:04354500122B97228C
:103E05008F2B90600263A20190702263A201AF2BF9
:103E1500122BA9E4F562F563852B6590702263A2E8
:103E2500019011C663A201AF65AE64AD63AC6212C9
:103E35002BDC8F658E648D638C627422252BF58255
:103E4500E43470F583E563F07423252BF582E434BF
:103E550070F583E562F07422252BF582E43470F564
:103E650083E0FFA3E0906F20CFF0A3EFF0E52B24D4
:103E750002F560200A127E117F9112395C7E707FF7
:103E850022E4FBAD60123B177568FFD211C2992081
:053E950099FDD2992205
:101C9F00E55E655D605875F00DE55DA424E2F582A3
:101CAF00E5F0346BF583E02405F52BD3940E400C4F
:101CBF00200A357E117F9C12395C802C75F00DE562
:101CCF005DA424DEF582E5F0346BF58363A2017425
:101CDF00042566F582E43460F58363A201AF2B120D
:101CEF002BA9E52B2566F566055D535D3F2275F043
:101CFF0075E56AA42436F582E5F03468F583E07063
:101D0F0003021E06E55C705575F075E56AA4243A6A
:101D1F00F582E5F03468F583E02405F52BD3940EB6
:101D2F00400C200A357E117F9C12395C802C75F097
:101D3F0075E56AA42436F582E5F03468F58363A26D
:101D4F000174042566F582E43460F58363A201AF64
:101D5F002B122BA9E52B2566F566055C2275F07510
:101D6F00E56AA42439F582E5F03468F583E0540F71
:101D7F00FFE55CD39F506575F075E56AA4243AF5CD
:101D8F0082E5F03468F58375F00DE55C1223F2E01F
:101D9F002405F52BD3940E400C200A3D7E117F9C19
:101DAF0012395C803475F075E56AA42436F582E546
:101DBF00F03468F58375F00DE55C1223F263A20130
:101DCF0074042566F582E43460F58363A201AF2BBA
:101DDF00122BA9E52B2566F566055C22E4F55C75EB
:101DEF00F075E56AA42436F582E5F03468F583E4EE
:101DFF00F0056A536A0722056A536A07E55B656F48
:101E0F00605875F00DE56FA424BAF582E5F03461E2
:101E1F00F583E02405F52BD3940E400C200A357E74
:101E2F00117F9C12395C802C75F00DE56FA424B6E0
:101E3F00F582E5F03461F58363A20174042566F53C
:101E4F0082E43460F58363A201AF2B122BA9E52B3B
:101E5F002566F566056F536F7F22E56775F00DA454
:101E6F002403F582E43461F583E06067E56775F07C
:101E7F000DA42407F582E43461F583E02405F52BE6
:101E8F00D3940E400C200A347E117F9C12395C8053
:101E9F002BE56775F00DA42403F582E43461F58317
:101EAF0063A20174042566F582E43460F58363A2AE
:101EBF0001AF2B122BA9E52B2566F566E56775F0AB
:101ECF000DA42403F582E43461F583E4F005675330
:101EDF00670722056753670775F068E56EA424232B
:101EEF00F582E5F03471F58375F00DE55F1223F29D
:101EFF00E07003021F8775F068E56EA42427F58252
:101F0F00E5F03471F58375F00DE55F1223F2E024EF
:101F1F0005F52BD3940E400C200A3D7E117F9C12A9
:101F2F00395C803475F068E56EA42423F582E5F002
:101F3F003471F58375F00DE55F1223F263A201741E
:101F4F00042566F582E43460F58363A201AF2B129A
:101F5F002BA9E52B2566F56675F068E56EA424239D
:101F6F00F582E5F03471F58375F00DE55F1223F21C
:101F7F00E4F0055F535F0722055FE55FC3940840F8
:091F8F0008E4F55F056E536E07CE
:011F98002226
:102E2400300028C200906F1FE0601204F0E0D394D9
:102E3400F0400A9080007480F0C2AF80FE90616F11
:102E4400E004F09061B5E0600214F0E508B4010C10
:102E5400E4F508D211C2992099FDD299E50BD394D7
:102E6400644007C210E4F561F50B30110F90616FF7
:102E7400E0D39414400BC211D21C8005E490616F1E
:102E8400F020113EE508703A301937F528E528C3DB
:102E940095695010121C9FE5666009D394C85004CC
:102EA400052880E9E566601AE4906002F0A37419CD
:102EB400F0E5662402FF123E05E4F566906000F03A
:102EC400A3F0E56C7003022FC1F528E4F56CF562FC
:102ED400F563E528547FF565E52854802422F582BE
:102EE400E4346FF58363A2019011C663A201AF6558
:102EF400AE64AD63AC62122BDC8F658E648D638C23
:102F040062E52854802422F582E4346FAF82F529E7
:102F14008F2A53287FE56345626022300A03022F1B
:102F2400C17E117FA712395CE4FBAD28AF2AAE291C
:102F3400123B177D03AF63AE62123A3D22200A2E84
:102F4400906170E0640160147E117FB212395CE418
:102F5400FBAD28AF2AAE29123B1780127E117FB732
:102F640012395CE4FBAD28AF2AAE29123B17E528E1
:102F7400B40408E490616DF0C21B22852A8285297D
:102F840083A3E024E7702CD215E52824FCF557C36D
:102F9400940E501BE52A2402FFE43529F5838F8221
:102FA40063A201907AF463A201AF57122BA922E421
:0D2FB400F55722200A077E117FC112395CFB
:012FC10022ED
:103F3400020881E493A3F8E493A34003F68001F21A
:103F440008DFF48029E493A3F85407240CC8C3338E
:103F5400C4540F4420C8834004F456800146F6DF5D
:103F6400E4800B01020408102040809048FDE47EA8
:103F7400019360BCA3FF543F30E509541FFEE49352
:103F8400A360010ECF54C025E060A840B8E493A319
:103F9400FAE493A3F8E493A3C8C582C8CAC583CA44
:103FA400F0A3C8C582C8CAC583CADFE9DEE780BEFC
:0149030000B3
:10226C00BB010689828A83E0225002E722BBFE0270
:09227C00E32289828A83E49322A3
:10228500BB010CE58229F582E5833AF583E022500E
:1022950006E92582F8E622BBFE06E92582F8E22258
:0D22A500E58229F582E5833AF583E4932272
:1022B200A3F8E0C5F025F0F0E582158270021583DF
:0622C200E0C838F0E8223C
:1022C80075F008758200EF2FFFEE33FECD33CDCCCD
:1022D80033CCC58233C5829BED9AEC99E582984050
:1022E8000CF582EE9BFEED9AFDEC99FC0FD5F0D62D
:1022F800E4CEFBE4CDFAE4CCF9A88222B800C1B957
:102308000059BA002DEC8BF084CFCECDFCE5F0CB94
:10231800F97818EF2FFFEE33FEED33FDEC33FCEBCD
:1023280033FB10D703994004EB99FB0FD8E5E4F988
:10233800FA227818EF2FFFEE33FEED33FDEC33FC75
:10234800C933C910D7059BE99A4007EC9BFCE99A69
:10235800F90FD8E0E4C9FAE4CCFB2275F010EF2FAE
:10236800FFEE33FEED33FDCC33CCC833C810D707AE
:102378009BEC9AE899400AED9BFDEC9AFCE899F8E9
:0E2388000FD5F0DAE4CDFBE4CCFAE4C8F9227C
:0E239600C3E49FFFE49EFEE49DFDE49CFC2258
:1023A400EB9FF5F0EA9E42F0E99D42F0E89C45F08F
:0123B4002206
:0C23B500ECF0A3EDF0A3EEF0A3EFF0229B
:1023C100A8828583F0D083D0821223D81223D81219
:1023D10023D81223D8E473E493A3C583C5F0C5833E
:1023E100C8C582C8F0A3C583C5F0C583C8C582C866
:0123F10022C9
:0C23F200A42582F582E5F03583F58322F6
:10194300E53B242FF8E6053B22782C302402782F40
:10195300E475F00112245F02226C201DEB7F2ED26E
:101963001D8018EF540F2490D43440D4FF30210B42
:10197300EF24BFB41A0050032461FFE53C60021555
:101983003C053FE53F7002053E30240D782CE4759D
:10199300F00112245FEF0223FE0245EA7403D2240E
:1019A3008003E4C224F53B8B2C8A2D892EE4F53C7D
:1019B300F53EF53FE53C60077F2012197E80F57503
:1019C3003DFFC21EC21DC21FC220C222C223C225A6
:1019D30012194CFF700D3024057F0012198FAF3F91
:1019E300AE3E22B4255FC2D5C22112194CFF24D0CA
:1019F300B40A00501A75F00A783C30D50508B6FFD2
:101A03000106C6A426F620D5047002D22080D9246C
:101A1300CFB41A00EF5004C2E5D221021B8FD21EAD
:101A230080C6D21D80C0D21F80BCD2D580BAD2223C
:101A330080B47F2012197E201F077401B53C00403B
:101A4300F1121943FF12197E0219B7D225D223804E
:101A530095121943FB121943FA121943F94A4B70B1
:101A63000679607A1C7BFF201F2EE53C602A7E00EE
:101A73008E8275830012228560060EEE653D70F03E
:101A8300C2D5EBC0E0EAC0E0E9C0E0EE121BD6D05D
:101A9300E0F9D0E0FAD0E0FB12226CFF60AAEBC0C1
:101AA300E0EAC0E0E9C0E012197ED0E02401F9D0F9
:101AB300E03400FAD0E0FBE53D0460DCD53DD9809D
:101AC300877BFF7A1B79D2D21F809C7910800279A1
:101AD30008C223C2258008D2D5790A8004790AC2B4
:101AE300D5E53D047002F53DE4FAFDFEFF1219430E
:101AF300FC7B08201E13121943FD7B10301D0A12B4
:101B03001943FE121943FF7B20EC3382D592D55043
:101B130013C3E4301D069FFFE49EFEE4201E039DD5
:101B2300FDE49CFCE4CBF8C21EEC700CCFCECDCC14
:101B3300E824F8F870F38017C3EF33FFEE33FEEDBC
:101B430033FDEC33FCEB33FB994002FB0FD8E9EB9D
:101B5300301E05F8D0E0C448B21EC0E00AEC4D4E7A
:101B63004F78207B0070C2EAB53D0040BCC0E01254
:101B73001BD8D0F0D0E0201E04C4C0E0C4B21EC005
:101B8300F0121967D0F0D5F0EB0219B71224BE1A80
:101B930054531ACE581A254C1A21421AD24F1ADA24
:0F1BA300441ADA491A3A431AE0551AC4461AC4CA
:101BB200451AC4471C80501A292D1A2D2E1A502B53
:101BC2001A31231A4E201C692A19E94800001A48C2
:101BD2003F3F3F00790AA2D5202014302209B910D4
:101BE200020404B9080104A2D520230250010420F2
:101BF2001F68921FB53C005034C0E07F203020198E
:101C02007F30A21F72237222500F121C2FC21FC2DA
:101C120023C222C2257F30800F302203E9C0E012A6
:101C2200197E302203D0E0F9D0E0B53CCC30221747
:101C32007F30B9100C12197E7F583021077F7880CF
:101C420003B9080312197E301F057F2D02197E7F0A
:101C5200202025F87F2B2023F322921F80CF286E8D
:101C6200756C6C2900D21E121943301EF8C21E7800
:101C72003C30D50108F60219E92D50434958121992
:101C8200432403B405004001E4901C7B9312196FB6
:0D1C9200743A12196FD220753C04021ACE6C
:102C80008B2C8A2D892EE4F538F537F536F535F598
:102C900033F534E5304531452F6012EBC0E0EAC032
:102CA000E0E9C0E0AB2FAA30A93112246FAB2C05AC
:102CB0002EE52EAA2D7002052D14F912226CF5397D
:102CC000C394094007E539D3940D40E1E539642008
:102CD00060DBE539B42D054334038016E539B42BA8
:102CE00005433401800C74FF252EF52E74FF352D1D
:102CF000F52DE53260046410703FAB2CAA2DA92E8F
:102D000012226C64306009E532702E75320A802917
:102D1000900001122285FF64786004EFB4581343D9
:102D200034017532107402252EF52EE4352DF52D63
:102D30008007E5327003753208AB2C052EE52EAA0C
:102D40002D7002052D14F912226CF539C3946140DF
:102D50000AE539D3947A50035339DF74D02539F515
:102D600039C3940A400CE5399411406D74F9253942
:102D7000F539E539D39532506043340185383D85C6
:102D8000373C85363B85353AAF327E00E4FCFDABFF
:102D900038AA37A936A835122410C8ECC8C9EDC91D
:102DA000CAEECACBEFCBE4FCFDFEEB2539F538EEDD
:102DB0003AF537ED39F536EC38F535AF38AE37AD95
:102DC00036FCAB3DAA3CA93BA83AD31223A450033E
:102DD000022D39433404022D39E53420E003E48028
:102DE0002DE5304531452F601EAB2CE52E24FFF933
:102DF000E52D34FFFAEBC0E0EAC0E0E9C0E0AB2F1C
:102E0000AA30A93112246FE53430E20774FFFFFEC7
:102E1000FDFC22E534AF38AE37AD36AC3530E103DA
:042E200002239622D1
:1023FE00BB010689828A83F0225002F722BBFE01BE
:02240E00F322B7
:10241000E88FF0A4CC8BF0A42CFCE98EF0A42CFC6B
:102420008AF0EDA42CFCEA8EF0A4CDA8F08BF0A4E9
:102430002DCC3825F0FDE98FF0A42CCD35F0FCEB48
:102440008EF0A4FEA9F0EB8FF0A4CFC5F02ECD390D
:0F245000FEE43CFCEAA42DCE35F0FDE43CFC227A
:10245F00FAE6FB0808E6F925F0F618E6CA3AF6227E
:10246F00BB011A89828A83D0F0D0E0F8D0E0F9D08E
:10247F00E0FAD0E0FBE8C0E0C0F00224ED5016E92E
:10248F00F8D083D082D0E0F9D0E0FAD0E0FBC08260
:10249F00C0830224E4BBFE16E9F8D083D082D0E0DB
:0F24AF00F9D0E0FAD0E0FBC082C0830224F6220D
:1024BE00D083D082F8E4937012740193700DA3A3AD
:1024CE0093F8740193F5828883E4737402936860C1
:0624DE00EFA3A3A380DFC1
:0924E400EBF608EAF608E9F6221D
:0924ED00EBF0A3EAF0A3E9F022F0
:0924F600EBF208EAF208E9F22217
:00000001FF
